 jsound

 Timestamp is 6a163892 (Tue May 26 20:19:30 2026)

 Preferred load address is 10000000

 Start         Length     Name                   Class
 0001:00000000 00000020H .text$di                CODE
 0001:00000020 00003c4fH .text$mn                CODE
 0001:00003c6f 0000000aH .text$yd                CODE
 0002:00000000 00000140H .idata$5                DATA
 0002:00000140 00000008H .00cfg                  DATA
 0002:00000148 00000004H .CRT$XCA                DATA
 0002:0000014c 00000004H .CRT$XCU                DATA
 0002:00000150 00000004H .CRT$XCZ                DATA
 0002:00000154 00000004H .CRT$XIA                DATA
 0002:00000158 00000004H .CRT$XIZ                DATA
 0002:0000015c 00000004H .CRT$XPA                DATA
 0002:00000160 00000004H .CRT$XPZ                DATA
 0002:00000164 00000004H .CRT$XTA                DATA
 0002:00000168 00000008H .CRT$XTZ                DATA
 0002:0000016c 00000000H .gfids$y                DATA
 0002:00000170 00000550H .rdata                  DATA
 0002:000006c0 00000000H .rdata$CastGuardVftablesA DATA
 0002:000006c0 00000000H .rdata$CastGuardVftablesC DATA
 0002:000006c0 00000004H .rdata$sxdata           DATA
 0002:000006c4 000000b0H .rdata$voltmd           DATA
 0002:00000774 0000032cH .rdata$zzzdbg           DATA
 0002:00000aa0 00000004H .rtc$IAA                DATA
 0002:00000aa4 00000004H .rtc$IZZ                DATA
 0002:00000aa8 00000004H .rtc$TAA                DATA
 0002:00000aac 00000004H .rtc$TZZ                DATA
 0002:00000ab0 00000090H .xdata$x                DATA
 0002:00000b40 000009d0H .edata                  DATA
 0002:00001510 0000008cH .idata$2                DATA
 0002:0000159c 00000014H .idata$3                DATA
 0002:000015b0 00000140H .idata$4                DATA
 0002:000016f0 00000646H .idata$6                DATA
 0003:00000000 00000038H .data                   DATA
 0003:00000038 0000052cH .bss                    DATA
 0004:00000000 00000060H .rsrc$01                DATA
 0004:00000060 00000368H .rsrc$02                DATA

  Address         Publics by Value              Rva+Base       Lib:Object

 0000:00000000       ___AbsoluteZero            00000000     <absolute>
 0000:00000000       ___arm64x_extra_rfe_table  00000000     <absolute>
 0000:00000000       ___arm64x_extra_rfe_table_size 00000000     <absolute>
 0000:00000000       ___arm64x_native_entrypoint 00000000     <absolute>
 0000:00000000       ___arm64x_redirection_metadata 00000000     <absolute>
 0000:00000000       ___arm64x_redirection_metadata_count 00000000     <absolute>
 0000:00000000       ___dynamic_value_reloc_table 00000000     <absolute>
 0000:00000000       ___enclave_config          00000000     <absolute>
 0000:00000000       ___guard_check_icall_a64n_fptr 00000000     <absolute>
 0000:00000000       ___guard_eh_cont_count     00000000     <absolute>
 0000:00000000       ___guard_eh_cont_table     00000000     <absolute>
 0000:00000000       ___guard_fids_count        00000000     <absolute>
 0000:00000000       ___guard_fids_table        00000000     <absolute>
 0000:00000000       ___guard_iat_count         00000000     <absolute>
 0000:00000000       ___guard_iat_table         00000000     <absolute>
 0000:00000000       ___guard_longjmp_count     00000000     <absolute>
 0000:00000000       ___guard_longjmp_table     00000000     <absolute>
 0000:00000000       ___hybrid_auxiliary_iat    00000000     <absolute>
 0000:00000000       ___hybrid_auxiliary_iat_copy 00000000     <absolute>
 0000:00000000       ___hybrid_code_map         00000000     <absolute>
 0000:00000000       ___hybrid_code_map_count   00000000     <absolute>
 0000:00000000       ___x64_code_ranges_to_entry_points 00000000     <absolute>
 0000:00000000       ___x64_code_ranges_to_entry_points_count 00000000     <absolute>
 0000:00000001       ___safe_se_handler_count   00000001     <absolute>
 0000:00000100       ___guard_flags             00000100     <absolute>
 0000:00000000       ___ImageBase               10000000     <linker-defined>
 0001:00000020       _Java_com_sun_media_sound_MidiInDevice_nClose@16 10001020 f   MidiInDevice.obj
 0001:0000002d       _Java_com_sun_media_sound_MidiInDevice_nGetMessages@16 1000102d f   MidiInDevice.obj
 0001:0000020b       _Java_com_sun_media_sound_MidiInDevice_nGetTimeStamp@16 1000120b f   MidiInDevice.obj
 0001:0000020b       _Java_com_sun_media_sound_MidiOutDevice_nGetTimeStamp@16 1000120b f   MidiOutDevice.obj
 0001:00000229       _Java_com_sun_media_sound_MidiInDevice_nOpen@12 10001229 f   MidiInDevice.obj
 0001:00000270       _Java_com_sun_media_sound_MidiInDevice_nStart@16 10001270 f   MidiInDevice.obj
 0001:00000299       _Java_com_sun_media_sound_MidiInDevice_nStop@16 10001299 f   MidiInDevice.obj
 0001:000002a6       _Java_com_sun_media_sound_MidiInDeviceProvider_nGetDescription@12 100012a6 f   MidiInDeviceProvider.obj
 0001:00000316       _Java_com_sun_media_sound_MidiInDeviceProvider_nGetName@12 10001316 f   MidiInDeviceProvider.obj
 0001:00000386       _Java_com_sun_media_sound_MidiInDeviceProvider_nGetNumDevices@8 10001386 f   MidiInDeviceProvider.obj
 0001:0000038e       _Java_com_sun_media_sound_MidiInDeviceProvider_nGetVendor@12 1000138e f   MidiInDeviceProvider.obj
 0001:0000038e       _Java_com_sun_media_sound_MidiOutDeviceProvider_nGetVendor@12 1000138e f   MidiOutDeviceProvider.obj
 0001:000003fe       _Java_com_sun_media_sound_MidiInDeviceProvider_nGetVersion@12 100013fe f   MidiInDeviceProvider.obj
 0001:0000046e       _Java_com_sun_media_sound_MidiOutDevice_nClose@16 1000146e f   MidiOutDevice.obj
 0001:0000047b       _Java_com_sun_media_sound_MidiOutDevice_nOpen@12 1000147b f   MidiOutDevice.obj
 0001:000004b9       _Java_com_sun_media_sound_MidiOutDevice_nSendLongMessage@32 100014b9 f   MidiOutDevice.obj
 0001:0000050d       _Java_com_sun_media_sound_MidiOutDevice_nSendShortMessage@28 1000150d f   MidiOutDevice.obj
 0001:00000524       _Java_com_sun_media_sound_MidiOutDeviceProvider_nGetDescription@12 10001524 f   MidiOutDeviceProvider.obj
 0001:00000594       _Java_com_sun_media_sound_MidiOutDeviceProvider_nGetName@12 10001594 f   MidiOutDeviceProvider.obj
 0001:00000604       _Java_com_sun_media_sound_MidiOutDeviceProvider_nGetNumDevices@8 10001604 f   MidiOutDeviceProvider.obj
 0001:0000060c       _Java_com_sun_media_sound_MidiOutDeviceProvider_nGetVersion@12 1000160c f   MidiOutDeviceProvider.obj
 0001:0000067c       ??0Data@MidiIn_OpenHelper@@QAE@XZ 1000167c f   PLATFORM_API_WinOS_MidiIn.obj
 0001:000006c8       ??1Data@MidiIn_OpenHelper@@QAE@XZ 100016c8 f   PLATFORM_API_WinOS_MidiIn.obj
 0001:000006fe       ?MIDI_IN_PutMessage@@YGXPAUHMIDIIN__@@IIII@Z 100016fe f   PLATFORM_API_WinOS_MidiIn.obj
 0001:000007ad       ?ThreadProc@MidiIn_OpenHelper@@KGKPAX@Z 100017ad f   PLATFORM_API_WinOS_MidiIn.obj
 0001:000007f7       ?getMidiInCaps@@YAHHPAUtagMIDIINCAPSA@@PAH@Z 100017f7 f   PLATFORM_API_WinOS_MidiIn.obj
 0001:00000817       ?midiInOpen@MidiIn_OpenHelper@@SAIHPAUtag_MidiDeviceHandle@@@Z 10001817 f   PLATFORM_API_WinOS_MidiIn.obj
 0001:00000871       ?unprepareBuffers@@YAHPAUtag_MidiDeviceHandle@@@Z 10001871 f   PLATFORM_API_WinOS_MidiIn.obj
 0001:000008b2       _MIDI_IN_CloseDevice       100018b2 f   PLATFORM_API_WinOS_MidiIn.obj
 0001:00000905       _MIDI_IN_GetDeviceDescription 10001905 f   PLATFORM_API_WinOS_MidiIn.obj
 0001:00000905       _MIDI_IN_GetDeviceVendor   10001905 f   PLATFORM_API_WinOS_MidiIn.obj
 0001:00000905       _MIDI_OUT_GetDeviceVendor  10001905 f   PLATFORM_API_WinOS_MidiOut.obj
 0001:0000090b       _MIDI_IN_GetDeviceName     1000190b f   PLATFORM_API_WinOS_MidiIn.obj
 0001:00000966       _MIDI_IN_GetDeviceVersion  10001966 f   PLATFORM_API_WinOS_MidiIn.obj
 0001:000009ce       _MIDI_IN_GetErrorStr       100019ce f   PLATFORM_API_WinOS_MidiIn.obj
 0001:000009ef       _MIDI_IN_GetMessage        100019ef f   PLATFORM_API_WinOS_MidiIn.obj
 0001:00000a34       _MIDI_IN_GetNumDevices     10001a34 f   PLATFORM_API_WinOS_MidiIn.obj
 0001:00000a3a       _MIDI_IN_GetTimeStamp      10001a3a f   PLATFORM_API_WinOS_MidiIn.obj
 0001:00000a3a       _MIDI_OUT_GetTimeStamp     10001a3a f   PLATFORM_API_WinOS_MidiOut.obj
 0001:00000a3f       _MIDI_IN_OpenDevice        10001a3f f   PLATFORM_API_WinOS_MidiIn.obj
 0001:00000b38       _MIDI_IN_ReleaseMessage    10001b38 f   PLATFORM_API_WinOS_MidiIn.obj
 0001:00000b80       _MIDI_IN_StartDevice       10001b80 f   PLATFORM_API_WinOS_MidiIn.obj
 0001:00000bd3       _MIDI_IN_StopDevice        10001bd3 f   PLATFORM_API_WinOS_MidiIn.obj
 0001:00000c1f       ___local_stdio_printf_options 10001c1f f i PLATFORM_API_WinOS_MidiIn.obj
 0001:00000c25       __vsnprintf_l              10001c25 f i PLATFORM_API_WinOS_MidiIn.obj
 0001:00000c58       _sprintf                   10001c58 f i PLATFORM_API_WinOS_MidiIn.obj
 0001:00000c72       _MIDI_OUT_CloseDevice      10001c72 f   PLATFORM_API_WinOS_MidiOut.obj
 0001:00000d01       _MIDI_OUT_GetDeviceDescription 10001d01 f   PLATFORM_API_WinOS_MidiOut.obj
 0001:00000dab       _MIDI_OUT_GetDeviceName    10001dab f   PLATFORM_API_WinOS_MidiOut.obj
 0001:00000e06       _MIDI_OUT_GetDeviceVersion 10001e06 f   PLATFORM_API_WinOS_MidiOut.obj
 0001:00000e67       _MIDI_OUT_GetErrorStr      10001e67 f   PLATFORM_API_WinOS_MidiOut.obj
 0001:00000e88       _MIDI_OUT_GetNumDevices    10001e88 f   PLATFORM_API_WinOS_MidiOut.obj
 0001:00000e90       _MIDI_OUT_OpenDevice       10001e90 f   PLATFORM_API_WinOS_MidiOut.obj
 0001:00000f75       _MIDI_OUT_SendLongMessage  10001f75 f   PLATFORM_API_WinOS_MidiOut.obj
 0001:000010b7       _MIDI_OUT_SendShortMessage 100020b7 f   PLATFORM_API_WinOS_MidiOut.obj
 0001:000010d2       _freeLongBuffer            100020d2 f   PLATFORM_API_WinOS_MidiOut.obj
 0001:0000112d       _freeLongBuffers           1000212d f   PLATFORM_API_WinOS_MidiOut.obj
 0001:0000116c       _getMidiOutCaps            1000216c f   PLATFORM_API_WinOS_MidiOut.obj
 0001:00001198       _unprepareLongBuffers      10002198 f   PLATFORM_API_WinOS_MidiOut.obj
 0001:000011df       _PORT_Close                100021df f   PLATFORM_API_WinOS_Ports.obj
 0001:0000124e       _PORT_GetControls          1000224e f   PLATFORM_API_WinOS_Ports.obj
 0001:00001471       _PORT_GetFloatValue        10002471 f   PLATFORM_API_WinOS_Ports.obj
 0001:0000150c       _PORT_GetIntValue          1000250c f   PLATFORM_API_WinOS_Ports.obj
 0001:00001552       _PORT_GetPortCount         10002552 f   PLATFORM_API_WinOS_Ports.obj
 0001:00001563       _PORT_GetPortMixerCount    10002563 f   PLATFORM_API_WinOS_Ports.obj
 0001:00001569       _PORT_GetPortMixerDescription 10002569 f   PLATFORM_API_WinOS_Ports.obj
 0001:000015f3       _PORT_GetPortName          100025f3 f   PLATFORM_API_WinOS_Ports.obj
 0001:0000163f       _PORT_GetPortType          1000263f f   PLATFORM_API_WinOS_Ports.obj
 0001:00001672       _PORT_Open                 10002672 f   PLATFORM_API_WinOS_Ports.obj
 0001:0000192c       _PORT_SetFloatValue        1000292c f   PLATFORM_API_WinOS_Ports.obj
 0001:000019eb       _PORT_SetIntValue          100029eb f   PLATFORM_API_WinOS_Ports.obj
 0001:00001a65       _addAllControls            10002a65 f   PLATFORM_API_WinOS_Ports.obj
 0001:00001a92       _componentType2type        10002a92 f   PLATFORM_API_WinOS_Ports.obj
 0001:00001af9       _createLineControls        10002af9 f   PLATFORM_API_WinOS_Ports.obj
 0001:00001c18       _createMuxControl          10002c18 f   PLATFORM_API_WinOS_Ports.obj
 0001:00001e0f       _createPortControl         10002e0f f   PLATFORM_API_WinOS_Ports.obj
 0001:00001f9f       _findDestLine              10002f9f f   PLATFORM_API_WinOS_Ports.obj
 0001:00001fc7       _getControlCount           10002fc7 f   PLATFORM_API_WinOS_Ports.obj
 0001:0000207c       _getControlInfo            1000307c f   PLATFORM_API_WinOS_Ports.obj
 0001:000020f2       _getControlValue           100030f2 f   PLATFORM_API_WinOS_Ports.obj
 0001:0000210f       _getDestinationCount       1000310f f   PLATFORM_API_WinOS_Ports.obj
 0001:00002147       _getFakeBalance            10003147 f   PLATFORM_API_WinOS_Ports.obj
 0001:000021d1       _getFakeVolume             100031d1 f   PLATFORM_API_WinOS_Ports.obj
 0001:00002217       _getMixerLineByDestination 10003217 f   PLATFORM_API_WinOS_Ports.obj
 0001:0000224c       _getMixerLineBySource      1000324c f   PLATFORM_API_WinOS_Ports.obj
 0001:00002288       _lineHasControls           10003288 f   PLATFORM_API_WinOS_Ports.obj
 0001:00002300       _setControlValue           10003300 f   PLATFORM_API_WinOS_Ports.obj
 0001:0000231d       _setFakeVolume             1000331d f   PLATFORM_API_WinOS_Ports.obj
 0001:000023b3       _MIDI_CreateLock           100033b3 f   PLATFORM_API_WinOS_Util.obj
 0001:000023ca       _MIDI_DestroyLock          100033ca f   PLATFORM_API_WinOS_Util.obj
 0001:000023e2       _MIDI_GetTimeStamp         100033e2 f   PLATFORM_API_WinOS_Util.obj
 0001:00002428       _MIDI_Lock                 10003428 f   PLATFORM_API_WinOS_Util.obj
 0001:0000243a       _MIDI_SetStartTime         1000343a f   PLATFORM_API_WinOS_Util.obj
 0001:00002452       _MIDI_Unlock               10003452 f   PLATFORM_API_WinOS_Util.obj
 0001:00002464       _MIDI_WinCreateEmptyLongBufferQueue 10003464 f   PLATFORM_API_WinOS_Util.obj
 0001:00002479       _MIDI_WinCreateLongBufferQueue 10003479 f   PLATFORM_API_WinOS_Util.obj
 0001:0000250a       _MIDI_WinDestroyLongBufferQueue 1000350a f   PLATFORM_API_WinOS_Util.obj
 0001:0000253a       _Java_com_sun_media_sound_Platform_nGetExtraLibraries@8 1000353a f   Platform.obj
 0001:0000254f       _Java_com_sun_media_sound_Platform_nGetLibraryForFeature@12 1000354f f   Platform.obj
 0001:00002571       _Java_com_sun_media_sound_Platform_nIsBigEndian@8 10003571 f   Platform.obj
 0001:00002579       _Java_com_sun_media_sound_Platform_nIsSigned8@8 10003579 f   Platform.obj
 0001:0000257e       _GetInternalErrorStr       1000357e f   PlatformMidi.obj
 0001:000025c7       _MIDI_CreateQueue          100035c7 f   PlatformMidi.obj
 0001:000025fe       _MIDI_DestroyQueue         100035fe f   PlatformMidi.obj
 0001:00002629       _MIDI_IN_InternalGetErrorString 10003629 f   PlatformMidi.obj
 0001:00002650       _MIDI_OUT_InternalGetErrorString 10003650 f   PlatformMidi.obj
 0001:00002677       _MIDI_QueueAddLong         10003677 f   PlatformMidi.obj
 0001:00002720       _MIDI_QueueAddShort        10003720 f   PlatformMidi.obj
 0001:000027a8       _MIDI_QueueClear           100037a8 f   PlatformMidi.obj
 0001:000027ce       _MIDI_QueueRead            100037ce f   PlatformMidi.obj
 0001:00002806       _MIDI_QueueRemove          10003806 f   PlatformMidi.obj
 0001:00002856       _Java_com_sun_media_sound_PortMixer_nClose@16 10003856 f   PortMixer.obj
 0001:0000286d       _Java_com_sun_media_sound_PortMixer_nControlGetFloatValue@16 1000386d f   PortMixer.obj
 0001:00002890       _Java_com_sun_media_sound_PortMixer_nControlGetIntValue@16 10003890 f   PortMixer.obj
 0001:000028ad       _Java_com_sun_media_sound_PortMixer_nControlSetFloatValue@20 100038ad f   PortMixer.obj
 0001:000028d1       _Java_com_sun_media_sound_PortMixer_nControlSetIntValue@20 100038d1 f   PortMixer.obj
 0001:000028ed       _Java_com_sun_media_sound_PortMixer_nGetControls@24 100038ed f   PortMixer.obj
 0001:00002973       _Java_com_sun_media_sound_PortMixer_nGetPortCount@16 10003973 f   PortMixer.obj
 0001:00002990       _Java_com_sun_media_sound_PortMixer_nGetPortName@20 10003990 f   PortMixer.obj
 0001:000029ed       _Java_com_sun_media_sound_PortMixer_nGetPortType@20 100039ed f   PortMixer.obj
 0001:00002a0f       _Java_com_sun_media_sound_PortMixer_nOpen@12 10003a0f f   PortMixer.obj
 0001:00002a1d       _PORT_AddControl           10003a1d f   PortMixer.obj
 0001:00002a49       _PORT_NewBooleanControl    10003a49 f   PortMixer.obj
 0001:00002ae2       _PORT_NewCompoundControl   10003ae2 f   PortMixer.obj
 0001:00002bbb       _PORT_NewFloatControl      10003bbb f   PortMixer.obj
 0001:00002ce9       _Java_com_sun_media_sound_PortMixerProvider_nGetNumDevices@8 10003ce9 f   PortMixerProvider.obj
 0001:00002cf1       _Java_com_sun_media_sound_PortMixerProvider_nNewPortMixerInfo@12 10003cf1 f   PortMixerProvider.obj
 0001:00002df8       _getPortMixerDescription   10003df8 f   PortMixerProvider.obj
 0001:00002e4d       _ThrowJavaMessageException 10003e4d f   Utilities.obj
 0001:00002e6d       _UTIL_IsBigEndianPlatform  10003e6d f   Utilities.obj
 0001:00002e6d       ___scrt_stub_for_is_c_termination_complete 10003e6d f   MSVCRT:ucrt_stubs.obj
 0001:00002e6d       __is_c_termination_complete 10003e6d f   MSVCRT:ucrt_stubs.obj
 0001:00002e70       @__security_check_cookie@4 10003e70 f   MSVCRT:secchk.obj
 0001:00002ec2       ___scrt_acquire_startup_lock 10003ec2 f   MSVCRT:utility.obj
 0001:00002ef4       ___scrt_dllmain_after_initialize_c 10003ef4 f   MSVCRT:utility.obj
 0001:00002f1f       ___scrt_dllmain_before_initialize_c 10003f1f f   MSVCRT:utility.obj
 0001:00002f2d       ___scrt_dllmain_crt_thread_attach 10003f2d f   MSVCRT:utility.obj
 0001:00002f4c       ___scrt_dllmain_crt_thread_detach 10003f4c f   MSVCRT:utility.obj
 0001:00002f59       ___scrt_dllmain_exception_filter 10003f59 f   MSVCRT:utility.obj
 0001:00002f8d       ___scrt_dllmain_uninitialize_c 10003f8d f   MSVCRT:utility.obj
 0001:00002fb0       ___scrt_dllmain_uninitialize_critical 10003fb0 f   MSVCRT:utility.obj
 0001:00002fbd       ___scrt_initialize_crt     10003fbd f   MSVCRT:utility.obj
 0001:00002ff6       ___scrt_initialize_onexit_tables 10003ff6 f   MSVCRT:utility.obj
 0001:0000307d       ___scrt_is_nonwritable_in_current_image 1000407d f   MSVCRT:utility.obj
 0001:00003111       ___scrt_release_startup_lock 10004111 f   MSVCRT:utility.obj
 0001:0000312e       ___scrt_uninitialize_crt   1000412e f   MSVCRT:utility.obj
 0001:00003156       __onexit                   10004156 f   MSVCRT:utility.obj
 0001:00003183       _atexit                    10004183 f   MSVCRT:utility.obj
 0001:000031a0       __ftol3                    100041a0 f   MSVCRT:ftol3.obj
 0001:00003210       __allmul                   10004210 f   MSVCRT:llmul.obj
 0001:00003584       __DllMainCRTStartup@12     10004584 f   MSVCRT:dll_dllmain.obj
 0001:000035a7       ___raise_securityfailure   100045a7 f   MSVCRT:gs_report.obj
 0001:000035cf       ___report_gsfailure        100045cf f   MSVCRT:gs_report.obj
 0001:000036c9       ___isa_available_init      100046c9 f   MSVCRT:cpu_disp.obj
 0001:0000389d       __get_startup_argv_mode    1000489d f   MSVCRT:argv_mode.obj
 0001:000038a1       ___scrt_is_ucrt_dll_in_use 100048a1 f   MSVCRT:ucrt_detection.obj
 0001:000038ad       ___scrt_fastfail           100048ad f   MSVCRT:utility_desktop.obj
 0001:000039c8       __crt_debugger_hook        100049c8 f   MSVCRT:utility_desktop.obj
 0001:000039d0       __SEH_prolog4              100049d0 f   MSVCRT:sehprolg4.obj
 0001:00003a15       __except_handler4          10004a15 f   MSVCRT:chandler4gs.obj
 0001:00003a44       @_guard_check_icall_nop@4  10004a44 f i MSVCRT:guard_support.obj
 0001:00003a94       ___security_init_cookie    10004a94 f   MSVCRT:gs_support.obj
 0001:00003adf       _DllMain@12                10004adf f   MSVCRT:dll_dllmain_stub.obj
 0001:00003b01       ?__scrt_initialize_type_info@@YAXXZ 10004b01 f   MSVCRT:tncleanup.obj
 0001:00003b0d       ?__scrt_uninitialize_type_info@@YAXXZ 10004b0d f   MSVCRT:tncleanup.obj
 0001:00003b19       ___local_stdio_scanf_options 10004b19 f i MSVCRT:default_local_stdio_options.obj
 0001:00003b1f       ___scrt_initialize_default_local_stdio_options 10004b1f f   MSVCRT:default_local_stdio_options.obj
 0001:00003b3c       ___scrt_get_dyn_tls_init_callback 10004b3c f   MSVCRT:dyn_tls_init.obj
 0001:00003b42       __RTC_Initialize           10004b42 f   MSVCRT:initsect.obj
 0001:00003b6e       __RTC_Terminate            10004b6e f   MSVCRT:initsect.obj
 0001:00003b9a       _memcpy                    10004b9a f   vcruntime:VCRUNTIME140.dll
 0001:00003ba0       _memset                    10004ba0 f   vcruntime:VCRUNTIME140.dll
 0001:00003ba6       __except_handler4_common   10004ba6 f   vcruntime:VCRUNTIME140.dll
 0001:00003bac       ___std_type_info_destroy_list 10004bac f   vcruntime:VCRUNTIME140.dll
 0001:00003bb2       _strcpy                    10004bb2 f   ucrt:api-ms-win-crt-string-l1-1-0.dll
 0001:00003bb8       __seh_filter_dll           10004bb8 f   ucrt:api-ms-win-crt-runtime-l1-1-0.dll
 0001:00003bbe       __configure_narrow_argv    10004bbe f   ucrt:api-ms-win-crt-runtime-l1-1-0.dll
 0001:00003bc4       __initialize_narrow_environment 10004bc4 f   ucrt:api-ms-win-crt-runtime-l1-1-0.dll
 0001:00003bca       __initialize_onexit_table  10004bca f   ucrt:api-ms-win-crt-runtime-l1-1-0.dll
 0001:00003bd0       __register_onexit_function 10004bd0 f   ucrt:api-ms-win-crt-runtime-l1-1-0.dll
 0001:00003bd6       __execute_onexit_table     10004bd6 f   ucrt:api-ms-win-crt-runtime-l1-1-0.dll
 0001:00003bdc       __crt_atexit               10004bdc f   ucrt:api-ms-win-crt-runtime-l1-1-0.dll
 0001:00003be2       __cexit                    10004be2 f   ucrt:api-ms-win-crt-runtime-l1-1-0.dll
 0001:00003be8       __initterm                 10004be8 f   ucrt:api-ms-win-crt-runtime-l1-1-0.dll
 0001:00003bee       __initterm_e               10004bee f   ucrt:api-ms-win-crt-runtime-l1-1-0.dll
 0001:00003bf4       ___acrt_initialize         10004bf4 f   MSVCRT:ucrt_stubs.obj
 0001:00003bf4       ___acrt_thread_attach      10004bf4 f   MSVCRT:ucrt_stubs.obj
 0001:00003bf4       ___acrt_thread_detach      10004bf4 f   MSVCRT:ucrt_stubs.obj
 0001:00003bf4       ___acrt_uninitialize       10004bf4 f   MSVCRT:ucrt_stubs.obj
 0001:00003bf4       ___acrt_uninitialize_critical 10004bf4 f   MSVCRT:ucrt_stubs.obj
 0001:00003bf4       ___scrt_stub_for_acrt_initialize 10004bf4 f   MSVCRT:ucrt_stubs.obj
 0001:00003bf4       ___scrt_stub_for_acrt_thread_attach 10004bf4 f   MSVCRT:ucrt_stubs.obj
 0001:00003bf4       ___scrt_stub_for_acrt_thread_detach 10004bf4 f   MSVCRT:ucrt_stubs.obj
 0001:00003bf4       ___scrt_stub_for_acrt_uninitialize 10004bf4 f   MSVCRT:ucrt_stubs.obj
 0001:00003bf4       ___scrt_stub_for_acrt_uninitialize_critical 10004bf4 f   MSVCRT:ucrt_stubs.obj
 0001:00003bf4       ___vcrt_initialize         10004bf4 f   MSVCRT:ucrt_stubs.obj
 0001:00003bf4       ___vcrt_thread_attach      10004bf4 f   MSVCRT:ucrt_stubs.obj
 0001:00003bf4       ___vcrt_thread_detach      10004bf4 f   MSVCRT:ucrt_stubs.obj
 0001:00003bf4       ___vcrt_uninitialize       10004bf4 f   MSVCRT:ucrt_stubs.obj
 0001:00003bf4       ___vcrt_uninitialize_critical 10004bf4 f   MSVCRT:ucrt_stubs.obj
 0001:00003bf7       __filter_x86_sse2_floating_point_exception 10004bf7 f   MSVCRT:x86_exception_filter.obj
 0001:00003bf7       __filter_x86_sse2_floating_point_exception_default 10004bf7 f   MSVCRT:x86_exception_filter.obj
 0002:00000000       __imp__SetUnhandledExceptionFilter@4 10005000     kernel32:KERNEL32.dll
 0002:00000004       __imp__InitializeCriticalSection@4 10005004     kernel32:KERNEL32.dll
 0002:00000008       __imp__EnterCriticalSection@4 10005008     kernel32:KERNEL32.dll
 0002:0000000c       __imp__LeaveCriticalSection@4 1000500c     kernel32:KERNEL32.dll
 0002:00000010       __imp__SetEvent@4          10005010     kernel32:KERNEL32.dll
 0002:00000014       __imp__WaitForSingleObject@8 10005014     kernel32:KERNEL32.dll
 0002:00000018       __imp__CreateEventA@16     10005018     kernel32:KERNEL32.dll
 0002:0000001c       __imp__InitializeSListHead@4 1000501c     kernel32:KERNEL32.dll
 0002:00000020       __imp__DisableThreadLibraryCalls@4 10005020     kernel32:KERNEL32.dll
 0002:00000024       __imp__GetSystemTimeAsFileTime@4 10005024     kernel32:KERNEL32.dll
 0002:00000028       __imp__GetCurrentThreadId@0 10005028     kernel32:KERNEL32.dll
 0002:0000002c       __imp__GetCurrentProcessId@0 1000502c     kernel32:KERNEL32.dll
 0002:00000030       __imp__QueryPerformanceCounter@4 10005030     kernel32:KERNEL32.dll
 0002:00000034       __imp__IsDebuggerPresent@0 10005034     kernel32:KERNEL32.dll
 0002:00000038       __imp__IsProcessorFeaturePresent@4 10005038     kernel32:KERNEL32.dll
 0002:0000003c       __imp__TerminateProcess@8  1000503c     kernel32:KERNEL32.dll
 0002:00000040       __imp__GetCurrentProcess@0 10005040     kernel32:KERNEL32.dll
 0002:00000044       __imp__UnhandledExceptionFilter@4 10005044     kernel32:KERNEL32.dll
 0002:00000048       __imp__DeleteCriticalSection@4 10005048     kernel32:KERNEL32.dll
 0002:0000004c       __imp__CreateThread@24     1000504c     kernel32:KERNEL32.dll
 0002:00000050       __imp__Sleep@4             10005050     kernel32:KERNEL32.dll
 0002:00000054       __imp__CloseHandle@4       10005054     kernel32:KERNEL32.dll
 0002:00000058       \177KERNEL32_NULL_THUNK_DATA 10005058     kernel32:KERNEL32.dll
 0002:0000005c       __imp___except_handler4_common 1000505c     vcruntime:VCRUNTIME140.dll
 0002:00000060       __imp__memset              10005060     vcruntime:VCRUNTIME140.dll
 0002:00000064       __imp__memcpy              10005064     vcruntime:VCRUNTIME140.dll
 0002:00000068       __imp____std_type_info_destroy_list 10005068     vcruntime:VCRUNTIME140.dll
 0002:0000006c       \177VCRUNTIME140_NULL_THUNK_DATA 1000506c     vcruntime:VCRUNTIME140.dll
 0002:00000070       __imp__mixerSetControlDetails@12 10005070     winmm:WINMM.dll
 0002:00000074       __imp__mixerGetControlDetailsA@12 10005074     winmm:WINMM.dll
 0002:00000078       __imp__mixerGetLineControlsA@12 10005078     winmm:WINMM.dll
 0002:0000007c       __imp__mixerGetLineInfoA@12 1000507c     winmm:WINMM.dll
 0002:00000080       __imp__mixerClose@4        10005080     winmm:WINMM.dll
 0002:00000084       __imp__mixerOpen@20        10005084     winmm:WINMM.dll
 0002:00000088       __imp__mixerGetDevCapsA@12 10005088     winmm:WINMM.dll
 0002:0000008c       __imp__mixerGetNumDevs@0   1000508c     winmm:WINMM.dll
 0002:00000090       __imp__timeEndPeriod@4     10005090     winmm:WINMM.dll
 0002:00000094       __imp__timeBeginPeriod@4   10005094     winmm:WINMM.dll
 0002:00000098       __imp__midiOutReset@4      10005098     winmm:WINMM.dll
 0002:0000009c       __imp__midiOutLongMsg@12   1000509c     winmm:WINMM.dll
 0002:000000a0       __imp__midiInGetNumDevs@0  100050a0     winmm:WINMM.dll
 0002:000000a4       __imp__midiOutShortMsg@8   100050a4     winmm:WINMM.dll
 0002:000000a8       __imp__midiOutUnprepareHeader@12 100050a8     winmm:WINMM.dll
 0002:000000ac       __imp__midiOutPrepareHeader@12 100050ac     winmm:WINMM.dll
 0002:000000b0       __imp__midiOutClose@4      100050b0     winmm:WINMM.dll
 0002:000000b4       __imp__midiOutOpen@20      100050b4     winmm:WINMM.dll
 0002:000000b8       __imp__midiOutGetErrorTextA@12 100050b8     winmm:WINMM.dll
 0002:000000bc       __imp__midiOutGetDevCapsA@12 100050bc     winmm:WINMM.dll
 0002:000000c0       __imp__midiOutGetNumDevs@0 100050c0     winmm:WINMM.dll
 0002:000000c4       __imp__midiInReset@4       100050c4     winmm:WINMM.dll
 0002:000000c8       __imp__midiInStop@4        100050c8     winmm:WINMM.dll
 0002:000000cc       __imp__midiInStart@4       100050cc     winmm:WINMM.dll
 0002:000000d0       __imp__midiInAddBuffer@12  100050d0     winmm:WINMM.dll
 0002:000000d4       __imp__midiInUnprepareHeader@12 100050d4     winmm:WINMM.dll
 0002:000000d8       __imp__midiInPrepareHeader@12 100050d8     winmm:WINMM.dll
 0002:000000dc       __imp__midiInClose@4       100050dc     winmm:WINMM.dll
 0002:000000e0       __imp__midiInOpen@20       100050e0     winmm:WINMM.dll
 0002:000000e4       __imp__midiInGetErrorTextA@12 100050e4     winmm:WINMM.dll
 0002:000000e8       __imp__midiInGetDevCapsA@12 100050e8     winmm:WINMM.dll
 0002:000000ec       __imp__timeGetTime@0       100050ec     winmm:WINMM.dll
 0002:000000f0       \177WINMM_NULL_THUNK_DATA  100050f0     winmm:WINMM.dll
 0002:000000f4       __imp__malloc              100050f4     ucrt:api-ms-win-crt-heap-l1-1-0.dll
 0002:000000f8       __imp__free                100050f8     ucrt:api-ms-win-crt-heap-l1-1-0.dll
 0002:000000fc       \177api-ms-win-crt-heap-l1-1-0_NULL_THUNK_DATA 100050fc     ucrt:api-ms-win-crt-heap-l1-1-0.dll
 0002:00000100       __imp___seh_filter_dll     10005100     ucrt:api-ms-win-crt-runtime-l1-1-0.dll
 0002:00000104       __imp___configure_narrow_argv 10005104     ucrt:api-ms-win-crt-runtime-l1-1-0.dll
 0002:00000108       __imp___initialize_narrow_environment 10005108     ucrt:api-ms-win-crt-runtime-l1-1-0.dll
 0002:0000010c       __imp___initialize_onexit_table 1000510c     ucrt:api-ms-win-crt-runtime-l1-1-0.dll
 0002:00000110       __imp___register_onexit_function 10005110     ucrt:api-ms-win-crt-runtime-l1-1-0.dll
 0002:00000114       __imp___execute_onexit_table 10005114     ucrt:api-ms-win-crt-runtime-l1-1-0.dll
 0002:00000118       __imp___cexit              10005118     ucrt:api-ms-win-crt-runtime-l1-1-0.dll
 0002:0000011c       __imp___crt_atexit         1000511c     ucrt:api-ms-win-crt-runtime-l1-1-0.dll
 0002:00000120       __imp___initterm           10005120     ucrt:api-ms-win-crt-runtime-l1-1-0.dll
 0002:00000124       __imp___initterm_e         10005124     ucrt:api-ms-win-crt-runtime-l1-1-0.dll
 0002:00000128       \177api-ms-win-crt-runtime-l1-1-0_NULL_THUNK_DATA 10005128     ucrt:api-ms-win-crt-runtime-l1-1-0.dll
 0002:0000012c       __imp____stdio_common_vsprintf 1000512c     ucrt:api-ms-win-crt-stdio-l1-1-0.dll
 0002:00000130       \177api-ms-win-crt-stdio-l1-1-0_NULL_THUNK_DATA 10005130     ucrt:api-ms-win-crt-stdio-l1-1-0.dll
 0002:00000134       __imp__strcpy              10005134     ucrt:api-ms-win-crt-string-l1-1-0.dll
 0002:00000138       __imp__strncpy             10005138     ucrt:api-ms-win-crt-string-l1-1-0.dll
 0002:0000013c       \177api-ms-win-crt-string-l1-1-0_NULL_THUNK_DATA 1000513c     ucrt:api-ms-win-crt-string-l1-1-0.dll
 0002:00000140       ___guard_check_icall_fptr  10005140     MSVCRT:guard_support.obj
 0002:00000144       ___castguard_check_failure_os_handled_fptr 10005144     MSVCRT:guard_support.obj
 0002:00000148       ___xc_a                    10005148     MSVCRT:initializers.obj
 0002:00000150       ___xc_z                    10005150     MSVCRT:initializers.obj
 0002:00000154       ___xi_a                    10005154     MSVCRT:initializers.obj
 0002:00000158       ___xi_z                    10005158     MSVCRT:initializers.obj
 0002:0000015c       ___xp_a                    1000515c     MSVCRT:initializers.obj
 0002:00000160       ___xp_z                    10005160     MSVCRT:initializers.obj
 0002:00000164       ___xt_a                    10005164     MSVCRT:initializers.obj
 0002:00000168       ___xt_z                    10005168     MSVCRT:initializers.obj
 0002:00000170       ??_C@_0CK@BNIEGIBB@javax?1sound?1midi?1MidiUnavailabl@ 10005170     MidiInDevice.obj
 0002:0000019c       ??_C@_05NPPFNMNL@?$CIIJ?$CJV@ 1000519c     MidiInDevice.obj
 0002:000001a4       ??_C@_0BF@LEBFAHIB@callbackShortMessage@ 100051a4     MidiInDevice.obj
 0002:000001bc       ??_C@_06PFGPJLID@?$CI?$FLBJ?$CJV@ 100051bc     MidiInDevice.obj
 0002:000001c4       ??_C@_0BE@CLHHHCK@callbackLongMessage@ 100051c4     MidiInDevice.obj
 0002:000001d8       ??_C@_0N@JNOBNNBP@Unknown?5name@ 100051d8     MidiInDeviceProvider.obj
 0002:000001e8       ??_C@_0P@FLAGCHHF@Unknown?5vendor@ 100051e8     MidiInDeviceProvider.obj
 0002:000001f8       ??_C@_0BF@LIAFPILD@No?5details?5available@ 100051f8     MidiInDeviceProvider.obj
 0002:00000210       ??_C@_0BA@EMALCDDA@Unknown?5version@ 10005210     MidiInDeviceProvider.obj
 0002:00000220       ??_C@_05KBEOJPB@?$CFd?4?$CFd@ 10005220     PLATFORM_API_WinOS_MidiIn.obj
 0002:00000228       ??_C@_0BD@GIDICAOP@External?5MIDI?5Port@ 10005228     PLATFORM_API_WinOS_MidiOut.obj
 0002:0000023c       ??_C@_0CB@BKPHBOPD@Internal?5square?5wave?5synthesize@ 1000523c     PLATFORM_API_WinOS_MidiOut.obj
 0002:00000260       ??_C@_0BI@BENILECD@Internal?5FM?5synthesizer@ 10005260     PLATFORM_API_WinOS_MidiOut.obj
 0002:00000278       ??_C@_0BP@HFJPHHGA@Internal?5synthesizer?5?$CIgeneric?$CJ@ 10005278     PLATFORM_API_WinOS_MidiOut.obj
 0002:00000298       ??_C@_0BE@GKHJJDH@Windows?5MIDI_MAPPER@ 10005298     PLATFORM_API_WinOS_MidiOut.obj
 0002:000002ac       ??_C@_0BO@JHOFOEDM@Internal?5software?5synthesizer@ 100052ac     PLATFORM_API_WinOS_MidiOut.obj
 0002:000002cc       ??_C@_0L@CPKCBHCN@Port?5Mixer@ 100052cc     PLATFORM_API_WinOS_Ports.obj
 0002:000002d7       ??_C@_00CNPNBAHC@@         100052d7     PLATFORM_API_WinOS_Ports.obj
 0002:000002d8       __real@3f000000            100052d8     PLATFORM_API_WinOS_Ports.obj
 0002:000002dc       __real@3f800000            100052dc     PLATFORM_API_WinOS_Ports.obj
 0002:000002e0       __real@40000000            100052e0     PLATFORM_API_WinOS_Ports.obj
 0002:000002e4       __real@bf800000            100052e4     PLATFORM_API_WinOS_Ports.obj
 0002:000002f0       __xmm@41f00000000000000000000000000000 100052f0     PLATFORM_API_WinOS_Ports.obj
 0002:00000300       ??_C@_08NPPDGNH@jsoundds@  10005300     Platform.obj
 0002:0000030c       ??_C@_0BG@PNPJGPKL@feature?5not?5supported@ 1000530c     PlatformMidi.obj
 0002:00000324       ??_C@_0BC@GOGOPKAK@invalid?5device?5ID@ 10005324     PlatformMidi.obj
 0002:00000338       ??_C@_0BP@CMLKCPDD@internal?5error?3?5invalid?5handle@ 10005338     PlatformMidi.obj
 0002:00000358       ??_C@_0O@BNNCBLEN@out?5of?5memory@ 10005358     PlatformMidi.obj
 0002:00000368       ??_C@_0CH@PANCBAOC@com?1sun?1media?1sound?1PortMixer$B@ 10005368     PortMixer.obj
 0002:00000390       ??_C@_0BH@DOGHFNPN@?$CIJLjava?1lang?1String?$DL?$CJV@ 10005390     PortMixer.obj
 0002:000003a8       ??_C@_06FALKBLGB@?$DMinit?$DO@ 100053a8     PortMixer.obj
 0002:000003b0       ??_C@_04IOCNJLNK@Mute@     100053b0     PortMixer.obj
 0002:000003b8       ??_C@_06HJGPBJLE@Select@   100053b8     PortMixer.obj
 0002:000003c0       ??_C@_0CH@ECCNHGI@com?1sun?1media?1sound?1PortMixer$C@ 100053c0     PortMixer.obj
 0002:000003e8       ??_C@_0DE@OMOINGJL@?$CILjava?1lang?1String?$DL?$FLLjavax?1soun@ 100053e8     PortMixer.obj
 0002:0000041c       ??_C@_0BM@GDMEENBL@javax?1sound?1sampled?1Control@ 1000541c     PortMixer.obj
 0002:00000438       ??_C@_0CI@OPKAAKLF@com?1sun?1media?1sound?1PortMixer$F@ 10005438     PortMixer.obj
 0002:00000460       ??_C@_0CM@PEFBHGMP@?$CIJLjava?1lang?1String?$DLFFFLjava?1la@ 10005460     PortMixer.obj
 0002:0000048c       ??_C@_0BL@HJNALIL@?$CIJIFFFLjava?1lang?1String?$DL?$CJV@ 1000548c     PortMixer.obj
 0002:000004a8       ??_C@_0BG@JLFLBLJI@?$CILjava?1lang?1Object?$DL?$CJV@ 100054a8     PortMixer.obj
 0002:000004c0       ??_C@_0L@MNLDOJKN@addElement@ 100054c0     PortMixer.obj
 0002:000004cc       ??_C@_0N@FMCAPCBL@Unknown?5Name@ 100054cc     PortMixerProvider.obj
 0002:000004dc       ??_C@_0P@JELLBOOJ@Unknown?5Vendor@ 100054dc     PortMixerProvider.obj
 0002:000004ec       ??_C@_0BA@LFHNEBGG@Unknown?5Version@ 100054ec     PortMixerProvider.obj
 0002:000004fc       ??_C@_0DE@HOKEHCEP@com?1sun?1media?1sound?1PortMixerPr@ 100054fc     PortMixerProvider.obj
 0002:00000530       ??_C@_0EN@JGCFGEEO@?$CIILjava?1lang?1String?$DLLjava?1lang?1@ 10005530     PortMixerProvider.obj
 0002:00000598       __pDefaultRawDllMain       10005598     MSVCRT:dll_dllmain.obj
 0002:00000598       __pRawDllMain              10005598     MSVCRT:dll_dllmain.obj
 0002:000005a8       __load_config_used         100055a8     MSVCRT:loadcfg.obj
 0002:000006c0       ___safe_se_handler_table   100056c0     <linker-defined>
 0002:000006c4       ___volatile_metadata       100056c4     <linker-defined>
 0002:00000aa0       ___rtc_iaa                 10005aa0     MSVCRT:initsect.obj
 0002:00000aa4       ___rtc_izz                 10005aa4     MSVCRT:initsect.obj
 0002:00000aa8       ___rtc_taa                 10005aa8     MSVCRT:initsect.obj
 0002:00000aac       ___rtc_tzz                 10005aac     MSVCRT:initsect.obj
 0002:00001510       __IMPORT_DESCRIPTOR_WINMM  10006510     winmm:WINMM.dll
 0002:00001524       __IMPORT_DESCRIPTOR_KERNEL32 10006524     kernel32:KERNEL32.dll
 0002:00001538       __IMPORT_DESCRIPTOR_VCRUNTIME140 10006538     vcruntime:VCRUNTIME140.dll
 0002:0000154c       __IMPORT_DESCRIPTOR_api-ms-win-crt-string-l1-1-0 1000654c     ucrt:api-ms-win-crt-string-l1-1-0.dll
 0002:00001560       __IMPORT_DESCRIPTOR_api-ms-win-crt-heap-l1-1-0 10006560     ucrt:api-ms-win-crt-heap-l1-1-0.dll
 0002:00001574       __IMPORT_DESCRIPTOR_api-ms-win-crt-stdio-l1-1-0 10006574     ucrt:api-ms-win-crt-stdio-l1-1-0.dll
 0002:00001588       __IMPORT_DESCRIPTOR_api-ms-win-crt-runtime-l1-1-0 10006588     ucrt:api-ms-win-crt-runtime-l1-1-0.dll
 0002:0000159c       __NULL_IMPORT_DESCRIPTOR   1000659c     winmm:WINMM.dll
 0003:00000000       ___security_cookie_complement 10007000     MSVCRT:gs_cookie.obj
 0003:00000004       ___security_cookie         10007004     MSVCRT:gs_cookie.obj
 0003:00000008       ___scrt_native_dllmain_reason 10007008     MSVCRT:utility.obj
 0003:00000010       __fltused                  10007010     MSVCRT:fltused.obj
 0003:00000020       ___isa_enabled             10007020     MSVCRT:cpu_disp.obj
 0003:00000030       ___scrt_ucrt_dll_is_in_use 10007030     MSVCRT:ucrt_stubs.obj
 0003:00000038       ?_OptionsStorage@?1??__local_stdio_printf_options@@9@4_KA 10007038     PLATFORM_API_WinOS_MidiIn.obj
 0003:00000040       ?data@MidiIn_OpenHelper@@1VData@1@A 10007040     PLATFORM_API_WinOS_MidiIn.obj
 0003:00000200       ___scrt_current_native_startup_state 10007200     MSVCRT:utility.obj
 0003:00000204       ___scrt_native_startup_lock 10007204     MSVCRT:utility.obj
 0003:00000544       ___isa_available           10007544     MSVCRT:cpu_disp.obj
 0003:00000548       ___favor                   10007548     MSVCRT:cpu_disp.obj
 0003:0000054c       ___scrt_debugger_hook_flag 1000754c     MSVCRT:utility_desktop.obj
 0003:00000550       ?__type_info_root_node@@3U__type_info_node@@A 10007550     MSVCRT:tncleanup.obj
 0003:00000558       ?_OptionsStorage@?1??__local_stdio_scanf_options@@9@4_KA 10007558     MSVCRT:default_local_stdio_options.obj
 0003:00000560       ___dyn_tls_init_callback   10007560     <common>

 entry point at        0001:00003584

 Static symbols

 0000:ffff6000       .debug$S                   10000000     jsound.exp
 0000:ffff6000       .debug$S                   10000000     vcruntime:VCRUNTIME140.dll
 0000:ffff6000       .debug$S                   10000000     vcruntime:VCRUNTIME140.dll
 0000:ffff6000       .debug$S                   10000000     vcruntime:VCRUNTIME140.dll
 0000:ffff6000       .debug$S                   10000000     vcruntime:VCRUNTIME140.dll
 0000:ffff6000       .debug$S                   10000000     vcruntime:VCRUNTIME140.dll
 0000:ffff6000       .debug$S                   10000000     vcruntime:VCRUNTIME140.dll
 0000:ffff6000       .debug$S                   10000000     ucrt:api-ms-win-crt-heap-l1-1-0.dll
 0000:ffff6000       .debug$S                   10000000     ucrt:api-ms-win-crt-heap-l1-1-0.dll
 0000:ffff6000       .debug$S                   10000000     ucrt:api-ms-win-crt-math-l1-1-0.dll
 0002:ffffb000       .idata$6                   10000000     ucrt:api-ms-win-crt-math-l1-1-0.dll
 0000:ffff6000       .debug$S                   10000000     ucrt:api-ms-win-crt-runtime-l1-1-0.dll
 0000:ffff6000       .debug$S                   10000000     ucrt:api-ms-win-crt-runtime-l1-1-0.dll
 0000:ffff6000       .debug$S                   10000000     ucrt:api-ms-win-crt-runtime-l1-1-0.dll
 0000:ffff6000       .debug$S                   10000000     ucrt:api-ms-win-crt-runtime-l1-1-0.dll
 0000:ffff6000       .debug$S                   10000000     ucrt:api-ms-win-crt-runtime-l1-1-0.dll
 0000:ffff6000       .debug$S                   10000000     ucrt:api-ms-win-crt-runtime-l1-1-0.dll
 0000:ffff6000       .debug$S                   10000000     ucrt:api-ms-win-crt-runtime-l1-1-0.dll
 0000:ffff6000       .debug$S                   10000000     ucrt:api-ms-win-crt-runtime-l1-1-0.dll
 0000:ffff6000       .debug$S                   10000000     ucrt:api-ms-win-crt-runtime-l1-1-0.dll
 0000:ffff6000       .debug$S                   10000000     ucrt:api-ms-win-crt-runtime-l1-1-0.dll
 0000:ffff6000       .debug$S                   10000000     ucrt:api-ms-win-crt-runtime-l1-1-0.dll
 0000:ffff6000       .debug$S                   10000000     ucrt:api-ms-win-crt-runtime-l1-1-0.dll
 0000:ffff6000       .debug$S                   10000000     ucrt:api-ms-win-crt-stdio-l1-1-0.dll
 0000:ffff6000       .debug$S                   10000000     ucrt:api-ms-win-crt-string-l1-1-0.dll
 0000:ffff6000       .debug$S                   10000000     ucrt:api-ms-win-crt-string-l1-1-0.dll
 0000:ffff6000       .debug$S                   10000000     kernel32:KERNEL32.dll
 0000:ffff6000       .debug$S                   10000000     kernel32:KERNEL32.dll
 0000:ffff6000       .debug$S                   10000000     kernel32:KERNEL32.dll
 0000:ffff6000       .debug$S                   10000000     kernel32:KERNEL32.dll
 0000:ffff6000       .debug$S                   10000000     kernel32:KERNEL32.dll
 0000:ffff6000       .debug$S                   10000000     kernel32:KERNEL32.dll
 0000:ffff6000       .debug$S                   10000000     kernel32:KERNEL32.dll
 0000:ffff6000       .debug$S                   10000000     kernel32:KERNEL32.dll
 0000:ffff6000       .debug$S                   10000000     kernel32:KERNEL32.dll
 0000:ffff6000       .debug$S                   10000000     kernel32:KERNEL32.dll
 0000:ffff6000       .debug$S                   10000000     kernel32:KERNEL32.dll
 0000:ffff6000       .debug$S                   10000000     kernel32:KERNEL32.dll
 0000:ffff6000       .debug$S                   10000000     kernel32:KERNEL32.dll
 0000:ffff6000       .debug$S                   10000000     kernel32:KERNEL32.dll
 0000:ffff6000       .debug$S                   10000000     kernel32:KERNEL32.dll
 0000:ffff6000       .debug$S                   10000000     kernel32:KERNEL32.dll
 0000:ffff6000       .debug$S                   10000000     kernel32:KERNEL32.dll
 0000:ffff6000       .debug$S                   10000000     kernel32:KERNEL32.dll
 0000:ffff6000       .debug$S                   10000000     kernel32:KERNEL32.dll
 0000:ffff6000       .debug$S                   10000000     kernel32:KERNEL32.dll
 0000:ffff6000       .debug$S                   10000000     kernel32:KERNEL32.dll
 0000:ffff6000       .debug$S                   10000000     kernel32:KERNEL32.dll
 0000:ffff6000       .debug$S                   10000000     kernel32:KERNEL32.dll
 0000:ffff6000       .debug$S                   10000000     kernel32:KERNEL32.dll
 0000:ffff6000       .debug$S                   10000000     winmm:WINMM.dll
 0000:ffff6000       .debug$S                   10000000     winmm:WINMM.dll
 0000:ffff6000       .debug$S                   10000000     winmm:WINMM.dll
 0000:ffff6000       .debug$S                   10000000     winmm:WINMM.dll
 0000:ffff6000       .debug$S                   10000000     winmm:WINMM.dll
 0000:ffff6000       .debug$S                   10000000     winmm:WINMM.dll
 0000:ffff6000       .debug$S                   10000000     winmm:WINMM.dll
 0000:ffff6000       .debug$S                   10000000     winmm:WINMM.dll
 0000:ffff6000       .debug$S                   10000000     winmm:WINMM.dll
 0000:ffff6000       .debug$S                   10000000     winmm:WINMM.dll
 0000:ffff6000       .debug$S                   10000000     winmm:WINMM.dll
 0000:ffff6000       .debug$S                   10000000     winmm:WINMM.dll
 0000:ffff6000       .debug$S                   10000000     winmm:WINMM.dll
 0000:ffff6000       .debug$S                   10000000     winmm:WINMM.dll
 0000:ffff6000       .debug$S                   10000000     winmm:WINMM.dll
 0000:ffff6000       .debug$S                   10000000     winmm:WINMM.dll
 0000:ffff6000       .debug$S                   10000000     winmm:WINMM.dll
 0000:ffff6000       .debug$S                   10000000     winmm:WINMM.dll
 0000:ffff6000       .debug$S                   10000000     winmm:WINMM.dll
 0000:ffff6000       .debug$S                   10000000     winmm:WINMM.dll
 0000:ffff6000       .debug$S                   10000000     winmm:WINMM.dll
 0000:ffff6000       .debug$S                   10000000     winmm:WINMM.dll
 0000:ffff6000       .debug$S                   10000000     winmm:WINMM.dll
 0000:ffff6000       .debug$S                   10000000     winmm:WINMM.dll
 0000:ffff6000       .debug$S                   10000000     winmm:WINMM.dll
 0000:ffff6000       .debug$S                   10000000     winmm:WINMM.dll
 0000:ffff6000       .debug$S                   10000000     winmm:WINMM.dll
 0000:ffff6000       .debug$S                   10000000     winmm:WINMM.dll
 0000:ffff6000       .debug$S                   10000000     winmm:WINMM.dll
 0000:ffff6000       .debug$S                   10000000     winmm:WINMM.dll
 0000:ffff6000       .debug$S                   10000000     winmm:WINMM.dll
 0000:ffff6000       .debug$S                   10000000     winmm:WINMM.dll
 0001:00000000       ??__E?data@MidiIn_OpenHelper@@1VData@1@A@@YAXXZ 10001000 f   PLATFORM_API_WinOS_MidiIn.obj
 0001:00002e7e       ?find_pe_section@@YAPAU_IMAGE_SECTION_HEADER@@QAEI@Z 10003e7e f   MSVCRT:utility.obj
 0001:000031a0       $$000000                   100041a0     MSVCRT:ftol3.obj
 0001:000031bf       _ftol3_default             100041bf     MSVCRT:ftol3.obj
 0001:000031d3       _ftol3_notsafe             100041d3     MSVCRT:ftol3.obj
 0001:000031f3       _ftol3_mincheck            100041f3     MSVCRT:ftol3.obj
 0001:000031f9       _ftol3_NaN                 100041f9     MSVCRT:ftol3.obj
 0001:00003201       _ftol3_retmin              10004201     MSVCRT:ftol3.obj
 0001:00003210       $$000000                   10004210     MSVCRT:llmul.obj
 0001:00003229       hard                       10004229     MSVCRT:llmul.obj
 0001:00003244       ?dllmain_crt_dispatch@@YGHQAUHINSTANCE__@@KQAX@Z 10004244 f   MSVCRT:dll_dllmain.obj
 0001:00003297       ?dllmain_crt_process_attach@@YAHQAUHINSTANCE__@@QAX@Z 10004297 f   MSVCRT:dll_dllmain.obj
 0001:0000339e       ?dllmain_crt_process_detach@@YAH_N@Z 1000439e f   MSVCRT:dll_dllmain.obj
 0001:0000344e       ?dllmain_dispatch@@YAHQAUHINSTANCE__@@KQAX@Z 1000444e f   MSVCRT:dll_dllmain.obj
 0001:00003559       ?dllmain_raw@@YGHQAUHINSTANCE__@@KQAX@Z 10004559 f   MSVCRT:dll_dllmain.obj
 0001:000039d0       $$000000                   100049d0     MSVCRT:sehprolg4.obj
 0001:00003a47       ___get_entropy             10004a47 f   MSVCRT:gs_support.obj
 0001:00003c6f       ??__F?data@MidiIn_OpenHelper@@1VData@1@A@@YAXXZ 10004c6f f   PLATFORM_API_WinOS_MidiIn.obj
 0002:0000014c       ??data$initializer$@MidiIn_OpenHelper@@1P6AXXZA@@3P6AXXZA 1000514c     PLATFORM_API_WinOS_MidiIn.obj
 0002:00000580       _NaN                       10005580     MSVCRT:ftol3.obj
 0002:00000584       _onept5                    10005584     MSVCRT:ftol3.obj
 0002:00000588       _DP2to32                   10005588     MSVCRT:ftol3.obj
 0002:00000588       _Int32ToUInt32             10005588     MSVCRT:ftol3.obj
 0002:0000059c       _GS_ExceptionPointers      1000559c     MSVCRT:gs_report.obj
 0002:00000ab0       __sehtable$___scrt_is_nonwritable_in_current_image 10005ab0     MSVCRT:utility.obj
 0002:00000ad0       __sehtable$?dllmain_crt_process_attach@@YAHQAUHINSTANCE__@@QAX@Z 10005ad0     MSVCRT:dll_dllmain.obj
 0002:00000af0       __sehtable$?dllmain_crt_process_detach@@YAH_N@Z 10005af0     MSVCRT:dll_dllmain.obj
 0002:00000b18       __sehtable$?dllmain_dispatch@@YAHQAUHINSTANCE__@@KQAX@Z 10005b18     MSVCRT:dll_dllmain.obj
 0002:00000b40       .edata                     10005b40     jsound.exp
 0002:00000b68       rgpv                       10005b68     jsound.exp
 0002:00000bfc       rgszName                   10005bfc     jsound.exp
 0002:00000c90       rgwOrd                     10005c90     jsound.exp
 0002:00000cda       szName                     10005cda     jsound.exp
 0002:00000ce5       $N00001                    10005ce5     jsound.exp
 0002:00000d27       $N00002                    10005d27     jsound.exp
 0002:00000d62       $N00003                    10005d62     jsound.exp
 0002:00000da2       $N00004                    10005da2     jsound.exp
 0002:00000ddf       $N00005                    10005ddf     jsound.exp
 0002:00000e1d       $N00006                    10005e1d     jsound.exp
 0002:00000e4e       $N00007                    10005e4e     jsound.exp
 0002:00000e85       $N00008                    10005e85     jsound.exp
 0002:00000ebd       $N00009                    10005ebd     jsound.exp
 0002:00000eed       $N00010                    10005eed     jsound.exp
 0002:00000f1e       $N00011                    10005f1e     jsound.exp
 0002:00000f4e       $N00012                    10005f4e     jsound.exp
 0002:00000f91       $N00013                    10005f91     jsound.exp
 0002:00000fcd       $N00014                    10005fcd     jsound.exp
 0002:0000100e       $N00015                    1000600e     jsound.exp
 0002:0000104c       $N00016                    1000604c     jsound.exp
 0002:0000108b       $N00017                    1000608b     jsound.exp
 0002:000010bd       $N00018                    100060bd     jsound.exp
 0002:000010f6       $N00019                    100060f6     jsound.exp
 0002:00001127       $N00020                    10006127     jsound.exp
 0002:00001163       $N00021                    10006163     jsound.exp
 0002:000011a0       $N00022                    100061a0     jsound.exp
 0002:000011d8       $N00023                    100061d8     jsound.exp
 0002:00001214       $N00024                    10006214     jsound.exp
 0002:00001246       $N00025                    10006246     jsound.exp
 0002:00001276       $N00026                    10006276     jsound.exp
 0002:000012b3       $N00027                    100062b3     jsound.exp
 0002:000012f4       $N00028                    100062f4     jsound.exp
 0002:00001322       $N00029                    10006322     jsound.exp
 0002:0000135f       $N00030                    1000635f     jsound.exp
 0002:0000139a       $N00031                    1000639a     jsound.exp
 0002:000013d7       $N00032                    100063d7     jsound.exp
 0002:00001412       $N00033                    10006412     jsound.exp
 0002:00001446       $N00034                    10006446     jsound.exp
 0002:0000147b       $N00035                    1000647b     jsound.exp
 0002:000014af       $N00036                    100064af     jsound.exp
 0002:000014e3       $N00037                    100064e3     jsound.exp
 0002:0000194a       .idata$6                   1000694a     winmm:WINMM.dll
 0002:00001b34       .idata$6                   10006b34     kernel32:KERNEL32.dll
 0002:00001b90       .idata$6                   10006b90     vcruntime:VCRUNTIME140.dll
 0002:00001cb2       .idata$6                   10006cb2     ucrt:api-ms-win-crt-string-l1-1-0.dll
 0002:00001cd4       .idata$6                   10006cd4     ucrt:api-ms-win-crt-heap-l1-1-0.dll
 0002:00001cf4       .idata$6                   10006cf4     ucrt:api-ms-win-crt-stdio-l1-1-0.dll
 0002:00001d14       .idata$6                   10006d14     ucrt:api-ms-win-crt-runtime-l1-1-0.dll
 0003:00000070       ?winMidiInErrMsg@@3PADA    10007070     PLATFORM_API_WinOS_MidiIn.obj
 0003:00000138       _winMidiOutErrMsg          10007138     PLATFORM_API_WinOS_MidiOut.obj
 0003:00000208       ?is_initialized_as_dll@@3_NA 10007208     MSVCRT:utility.obj
 0003:00000209       ?module_local_atexit_table_initialized@@3_NA 10007209     MSVCRT:utility.obj
 0003:0000020c       ?module_local_atexit_table@@3U_onexit_table_t@@A 1000720c     MSVCRT:utility.obj
 0003:00000218       ?module_local_at_quick_exit_table@@3U_onexit_table_t@@A 10007218     MSVCRT:utility.obj
 0003:00000224       ?__proc_attached@@3HA      10007224     MSVCRT:dll_dllmain.obj
 0003:00000228       _GS_ExceptionRecord        10007228     MSVCRT:gs_report.obj
 0003:00000278       _GS_ContextRecord          10007278     MSVCRT:gs_report.obj
 0004:00000060       $R000000                   10008060     jsound.dll.res
